:10000000B6012929B616B61EB61236190C28FE39C5
:10001000B700361503102429361A1428A600361600
:100020002B20031819282608322003181928B61E79
:1000300024292420492036113612B6113A088400AA
:100040003808841780042A283A0884003809800573
:100050008417800508001E204920242045203708E9
:10006000B6190138A2000830A300A20D03181E2003
:10007000031C242049204520A30B35281E2049209D
:100080003A08840038080005FF3E3B08840039091F
:1000900027283B0884003908800484173909800523
:1000A0002A28A400B7172730A3001030632003309C
:1000B000A300E8306320A30164306320A3010A3069
:1000C000632024086E28A2002508A1002408A000AF
:1000D00008212008031DB713B71B0800303EA700F6
:1000E0008611051205128316861105120512F030CD
:1000F000850583122708B6189B283A30A10098304E
:10010000CD203330A600B0201330A1008830CD20A0
:10011000B0206430CC20B0206430CC202230A60047
:10012000B02028309A200C309A2006309A20B6143D
:1001300027089B283614A600361CA9280512033C64
:10014000031CAE28AE200730A100D030CD20031410
:1001500008003614FE3C031924290516A60E361C89
:1001600036108615F030850526080F39850486116E
:10017000A60E3618B0283230CC2003140800A30194
:10018000A200FF30A207031CA307031C242903308D
:10019000A100DF30CD20C128A101E83EA000A109C7
:1001A000FC30031CD628A0070318D328A00764003E
:1001B000A10FD3282018DC28A01CE0280000E0288C
:1001C0000800A101A301A2000230F128A200013021
:1001D000F128A2000630F128A2000430F128A20084
:1001E0000530A80023082102031DF8282208200258
:1001F000043003180130031902302805031DFF30B5
:1002000024290038031DFF300405031DFF30242975
:10021000A501A4011030A600210DA40DA50D2208F2
:10022000A4022308031C230FA50203181E29220879
:10023000A40723080318230FA5070310A00DA10D81
:10024000A60B0C29200824298313031383126400AE
:10025000080007309F008316061186100610061648
:100260008616061732308312BF20C801BC01BD01BB
:100270000130C400C501A130BE00BF017030C6000E
:100280000630C7003130C000C101C201C3010610F1
:100290000330A300E830C020FE306F2001306F2013
:1002A0005A306F2045306F204B306F2045306F2023
:1002B00052306F2049306F2059306F2041306F200D
:1002C000FE306F20C0306F2059306F2041306F20DA
:1002D0005A306F2049306F2043306F2049306F20F3
:1002E0000330A300E830C020FE306F2001306F20C3
:1002F00079306F2061306F207A306F2069306F2045
:1003000063306F2069306F207A306F2040306F206B
:10031000FE306F20C0306F206D306F2079306F203D
:100320006E306F2065306F2074306F2063306F2027
:100330006F306F206D306F200330A300E830C02095
:10034000FE306F2001306F204108A5004008512089
:100350002C306F204308A500420851204D306F20FB
:1003600048306F207A306F206400061E242AC80AA5
:1003700064004808013C031DC3290130BC00BD01D5
:100380001430C400C5019630BF2064004808023C08
:10039000031DD0290A30BC00BD01C830C400C5010E
:1003A0009630BF2064004808033C031DDC29BC01D3
:1003B000BD010130C400C5019630BF206400043087
:1003C0004802031CE629BC01BD01C8013C08A0008D
:1003D0003D08A100A3010030EF20031D052AFE30D7
:1003E0006F20C0306F202B306F2020306F203530D1
:1003F0006F2030306F2020306F204B306F2048301E
:100400006F205A306F2020306F203C08A0003D083C
:10041000A100A3010030E920031D242AFE306F2033
:10042000C0306F203D08A5003C08512020306F20CF
:100430002B306F2020306F204D306F2048306F20E0
:100440005A306F2020306F200030861A0130A00013
:100450000130E120B2000030061B0130A000013065
:10046000E120B4003208840034080121B400B50052
:1004700064003408350403193F2A3230BF200030AD
:10048000861A0130A0000130E120B2000030061BC6
:100490000130A0000130E120B400320884003408AB
:1004A0000121B400B50064003408350403196A2B37
:1004B000A130BE00BF017030C6000630C700313029
:1004C000C000C101C201C301FE306F20C0306F20E7
:1004D00056306F2048306F2046306F2020306F201C
:1004E00034306F2039306F202D306F2031306F2045
:1004F00037306F2030306F2020306F204D306F202C
:1005000048306F205A306F2006100730A300D030DB
:10051000C0200030861A0130A0000130E120B20076
:100520000030061B0130A0000130E120B400320889
:10053000840034080121B400B50064003408350497
:1005400003196A2BA630BE00BF01B630C6000730C3
:10055000C7005830C000C101C201C301FE306F2086
:10056000C0306F2046306F204D306F2020306F201C
:1005700038306F2038306F202D306F2031306F20B1
:1005800030306F2038306F2020306F204D306F209A
:1005900048306F205A306F2006140730A300D03047
:1005A000C0200030861A0130A0000130E120B200E6
:1005B0000030061B0130A0000130E120B4003208F9
:1005C000840034080121B400B50064003408350407
:1005D00003196A2B9130BE00BF01E430C6000F3012
:1005E000C700AA30C000C101C201C301FE306F20A4
:1005F000C0306F2056306F2048306F2046306F205B
:1006000020306F2031306F2037306F2030306F2036
:100610002D306F2034306F2035306F2030306F2018
:1006200020306F204D306F2048306F205A306F20BF
:1006300006100730A300D030C0200030861A0130E9
:10064000A0000130E120B2000030061B0130A00004
:100650000130E120B4003208840034080121B400E4
:10066000B50064003408350403196A2B3830BE0025
:10067000BF01C430C6002530C700C230C000013001
:10068000C100C201C301FE306F20C0306F20553061
:100690006F2048306F2046306F2020306F2034307C
:1006A0006F2035306F2030306F202D306F20383084
:1006B0006F2035306F2035306F2020306F204D3067
:1006C0006F2048306F205A306F2006100730A3008B
:1006D000D030C0206400861E612D4408C60745083E
:1006E0000318013EC7073C08A0003D08A100A30174
:1006F0000030EF20031D8F2B3230C2070318C30ACE
:100700004208A0004308A1000330A300E830EF2016
:10071000031D8F2BC00A0319C10AC201C3013C0883
:10072000A0003D08A100A3010130EF20031D9B2B79
:10073000C00A0319C10A3C08A0003D08A100A3019A
:100740000A30EF20031DA82B0A30C0070318C10A86
:100750003E08A0003F08A100A301A130E320B200A1
:100760004008A0004108A100A301AA30E620B4007F
:100770003208840034080121B400B5006400340854
:1007800035040319F02BA130BE00BF017030C60044
:100790000630C7003130C000C101C201C301FE30C4
:1007A0006F20C0306F2056306F2048306F204630A9
:1007B0006F2020306F2034306F2039306F202D3083
:1007C0006F2031306F2037306F2030306F20203075
:1007D0006F204D306F2048306F205A306F20061048
:1007E0003E08A0003F08A100A301A630E320B2000C
:1007F0004008A0004108A100A3016C30E620B4002D
:100800003208840034080121B400B50064003408C3
:1008100035040319362CA630BE00BF01B630C60021
:100820000730C7005830C000C101C201C301FE300B
:100830006F20C0306F2046306F204D306F20203049
:100840006F2038306F2038306F202D306F203130DE
:100850006F2030306F2038306F2020306F204D30C7
:100860006F2048306F205A306F2006143E08A000D9
:100870003F08A100A3019130E320B2004008A0008E
:100880004108A1000130A300C230E620B4003208C4
:10089000840034080121B400B50064003408350434
:1008A0000319812C9130BE00BF01E430C6000F3027
:1008B000C700AA30C000C101C201C301FE306F20D1
:1008C000C0306F2056306F2048306F2046306F2088
:1008D00020306F2031306F2037306F2030306F2064
:1008E0002D306F2034306F2035306F2030306F2046
:1008F00020306F204D306F2048306F205A306F20ED
:1009000006103E08A0003F08A100A3013830E320F4
:10091000B2004008A0004108A1000330A3005730F6
:10092000E620B4003208840034080121B400B50088
:100930006400340835040319CD2C3830BE00BF01E3
:10094000C430C6002530C700C230C0000130C1002D
:10095000C201C301FE306F20C0306F2055306F20C0
:1009600048306F2046306F2020306F2034306F20A9
:1009700035306F2030306F202D306F2038306F20B1
:1009800035306F2035306F2020306F204D306F2094
:1009900048306F205A306F200610FE306F20013033
:1009A0006F204108A500400851202C306F204308DB
:1009B000A500420851204D306F2048306F207A301A
:1009C0006F20FE306F20C0306F2050306F204C30D1
:1009D0006F204C306F203A306F204708A500460842
:1009E00051203230BF203E08A0003F08A100A301E3
:1009F000A130EF20031D0E2D0630BA000230B800E2
:100A00000630BB000430B900C2300420470804207F
:100A100046080420CC300420A03002203E08A0006C
:100A20003F08A100A301A630EF20031D292D0630A9
:100A3000BA000230B8000630BB000430B900C23042
:100A400004204708042046080420CC300420A530A8
:100A500002203E08A0003F08A100A3019130EF2032
:100A6000031D442D0630BA000230B8000630BB002A
:100A70000430B900C230042047080420460804208E
:100A8000CC300420903002203E08A0003F08A10096
:100A9000A3013830EF20031D5F2D0630BA0002306D
:100AA000B8000630BB000430B900C230042047084B
:100AB000042046080420CC30042038300220963030
:100AC000BF206400061F632F4408A0004508A10052
:100AD000A3010130EF20031D862DFE306F20013071
:100AE0006F2054306F2041306F204E306F204930DE
:100AF0006F204D306F2053306F2049306F205A30B7
:100B00006F200430A300E230C020B4293C08A000CC
:100B10003D08A100A3010130EF20031D952D0130F8
:100B2000C0020030031C013EC1023C08A0003D0889
:100B3000A100A3010A30EF20031DA42D0A30C0023A
:100B40000030031C013EC1024408C6024508031CD4
:100B5000013EC7023E08A0003F08A100A301A1304A
:100B6000E320B2004008A0004108A100A3013130F9
:100B7000EC20B4003208840034080121B400B50030
:100B80006400340835040319F22DA130BE00BF0102
:100B9000E430C6000F30C700AA30C000C101C20156
:100BA000C301FE306F20C0306F2056306F204830B8
:100BB0006F2046306F2020306F2034306F20393066
:100BC0006F202D306F2031306F2037306F20303064
:100BD0006F2020306F204D306F2048306F205A300A
:100BE0006F2006103E08A0003F08A100A301A63018
:100BF000E320B2004008A0004108A100A301583042
:100C0000EC20B4003208840034080121B400B5009F
:100C10006400340835040319382EA630BE00BF0125
:100C20004630C6000930C7006C30C000C101C201A7
:100C3000C301FE306F20C0306F2046306F204D3032
:100C40006F2020306F2038306F2038306F202D30EB
:100C50006F2031306F2030306F2038306F202030DF
:100C60006F204D306F2048306F205A306F200614AF
:100C70003E08A0003F08A100A3019130E320B2008C
:100C80004008A0004108A100A301AA30EC20B40054
:100C90003208840034080121B400B500640034082F
:100CA00035040319832E9130BE00BF01C430C60045
:100CB0002530C700C230C0000130C100C201C301ED
:100CC000FE306F20C0306F2056306F2048306F20CC
:100CD00046306F2020306F2031306F2037306F204A
:100CE00030306F202D306F2034306F2035306F2042
:100CF00030306F2020306F204D306F2048306F2013
:100D00005A306F2006103E08A0003F08A100A30142
:100D10003830E320B2004008A0004108A1000130B3
:100D2000A300C230EC20B400320884003408012152
:100D3000B400B5006400340835040319CF2E3830F0
:100D4000BE00BF016830C6004530C7005730C00044
:100D50000330C100C201C301FE306F20C0306F20DC
:100D600055306F2048306F2046306F2020306F2084
:100D700034306F2035306F2030306F202D306F20B1
:100D800038306F2035306F2035306F2020306F20A5
:100D90004D306F2048306F205A306F200610FE30E3
:100DA0006F2001306F204108A500400851202C30F1
:100DB0006F204308A500420851204D306F20483075
:100DC0006F207A306F20FE306F20C0306F2050309F
:100DD0006F204C306F204C306F203A306F20470826
:100DE000A500460851203230BF203E08A0003F0831
:100DF000A100A301A130EF20031D102F0630BA007F
:100E00000230B8000630BB000430B900C230042004
:100E10004708042046080420CC300420A0300220DB
:100E20003E08A0003F08A100A301A630EF20031D4B
:100E30002B2F0630BA000230B8000630BB00043059
:100E4000B900C23004204708042046080420CC30F2
:100E50000420A53002203E08A0003F08A100A30105
:100E60009130EF20031D462F0630BA000230B80043
:100E70000630BB000430B900C2300420470804200B
:100E800046080420CC300420903002203E08A00008
:100E90003F08A100A3013830EF20031D612F063069
:100EA000BA000230B8000630BB000430B900C230CE
:100EB00004204708042046080420CC3004203830A1
:080EC00002209630BF20B42986
:02400E00653F0C
:00000001FF
